:020000040000FA
:02000000812855
:02000800AE2A1E
:10001000D10000300D28D1004030D20048207C3083
:10002000512052085120510851204D20182008001D
:100030000A30CC001B28CC0B1A28080028309A2242
:10004000383008203930082014300820703008205B
:10005000563008206C300820C8309A2238300820EA
:100060000C3008200130082001309A228D2208002F
:1000700044208A110A12D00A0319CF0A003E03193C
:1000800043280B20382808004F088A0050088200B7
:100090008514051405108510080085140510051435
:1000A0000800D3000830D4000510D31B05148514B4
:1000B0008510D30DD40B5428831605148312851490
:1000C0000000851083160510831208000830D40044
:1000D0008316051483128514031005180314D30D19
:1000E0008510D40B6B288316051083125308080063
:1000F0000510851485100514080005148514851055
:10010000080083018B0185010730990083163C307C
:10011000850034309700950070308F0008308100E2
:10012000831281018B128B170514851497221E20D0
:100130000C3008200230CB00803008200030CF0087
:10014000BD30D0003820C03008203820A822A82296
:10015000803008203820C03008203820A822A8226B
:10016000CB0B9C2801300820A822A822EA206F216E
:10017000C60146150930C500152946346D3453347F
:1001800074346534723465346F3400342034203470
:1001900052346134643469346F342034003456345A
:1001A00065347234203431342E34303434340034F5
:1001B00020346234793420344D342E345934203490
:1001C0000034203456346F346C343D3420342034C1
:1001D00020340034831626309B0083124330840081
:1001E0000230CB0083161C141A089B0A831280006D
:1001F000840ACB0BF2280800831626309B0083125A
:10020000433084000230CB00000883169A001C158E
:1002100055309D00AA309D009C149C180D299B0A06
:100220008312840ACB0B04290800851E3B21051E7E
:100230004821851D5521051D6121461C2C296F2152
:10024000461093228B120530C200383081002730CF
:10025000C0001030C1008B16461D36294908CF005A
:100260004A08D0004611C03008203820C61C152985
:10027000FC20C61015299322851A45294614C3036C
:10028000430A031D45294508C300851E452908006A
:100290009322051A52294614C30A4308450203183B
:1002A0005229C301051E52290800932285195E298F
:1002B0004614C403440A031D5E29C401851D5E293A
:1002C0000800932205196C294614C40A44080F3CFF
:1002D00003186C290F30C400051D6C29080001307B
:1002E000CF00AF30D0004308C9000310C90DC90DBD
:1002F0004908CA00C90D490D0318CF0A4A07031857
:10030000CF0AD0070318CF0A8030082038204F08C2
:10031000C9005008CA000930D0070318CF0A44208A
:10032000C700D00A0319CF0A4420C800C0300820F3
:100330000030CF00E130D00038200A3044020318EA
:10034000A529C63008204408AB29C5300820313023
:100350000B200A30440230380B20772208004E343C
:10036000413443344B343534203420342034003489
:100370002034373439342E3435344D3448347A34DB
:1003800000340834D83454344F344B3459344F3457
:10039000203446344D3400342034383430342E3454
:1003A00030344D3448347A3400340A3418344A3402
:1003B0002D345734413456344534203420340034FD
:1003C0002034383431342E3433344D3448347A3494
:1003D00000340D3458344E3448344B3420345934BE
:1003E0004B344834203400342034383431342E3403
:1003F00039344D3448347A3400340E34D8344E34E1
:1004000048344B34203454344B344F34203400348B
:100410002034383432342E3435344D3448347A3440
:1004200000341034583459344F344B344F3448343A
:1004300041344D34413400342034383434342E3493
:1004400037344D3448347A3400341534D834493490
:100450006E3474346534723446344D342034003490
:100460002034383439342E3437344D3448347A34E7
:100470000034223458345434423453342034463413
:100480004D342034203400342034393430342E3488
:1004900035344D3448347A340034243458344234BA
:1004A00055344E344B344134203446344D340034CA
:1004B0002034393431342E3436344D3448347A349F
:1004C0000034273418344E344934503450344F34C7
:1004D0004E342034203400342034393433342E3434
:1004E00030344D3448347A3400342A349834482037
:1004F00020305120D0305120013051204708512068
:1005000048085120003051200030512088305120BF
:100510004408803851204D2008002730CC00902A14
:10052000CC0B8F2A08001E309A2A64309A2AC830D1
:100530009A2A0130CD00DD30CC009E2A9F2AA02AC5
:10054000CC0B9D2A0000A42AA52ACD0B9B2A0800CB
:100550000A30CE009522CE0BAA2A0800F00003082C
:10056000F10083120B1DCE2A0B11383081000130AF
:10057000C1020319BF2A0318CE2AC002CE2AC0081E
:10058000031DCE2A2730C0001030C10005304202C2
:1005900003194615C20BCE2AC6148B1271088300AC
:0605A000F00E700E0900D0
:02400E00C43FAD
:1042000043006F0070007900720069006700680069
:1042100074002000280043002900200032003000F4
:10422000320030002D00320030003200310020001A
:104230006200790020004D002E00590061006D00E1
:1042400061006D006F0074006F00FF00030001004B
:00000001FF
